:100000008A110A1205280000090007309F00831694
:1000100086018501831206142030A0000330A10060
:100020000227D725D1233020AC012C08053C031C26
:100030002C28AD012D083B3C031C26280230A000D3
:10004000A10102270130AD07031C1A281F308305C8
:100050000130AC07031C15281F3083050B282F28FF
:10006000061086178616BC30A0000230A1000227B9
:100070009320A020A020A020932011211121112144
:100080009320AD012D08013C031C5328D9204121A8
:100090004921C120192119219921B920932001302A
:1000A000AD07031C42281F308305E120E920792198
:1000B00051211121F120932021211921292193205F
:1000C000612119219320B120E920012193201121E0
:1000D000D12029210121D920C120B120F120932054
:1000E0002121F920D1209320292121212921012119
:1000F0009320A020A020A02093200C220C220C22D0
:10010000A121A521AC21BB21D221E121E121EE21B8
:10011000FF21A1216122F430A0000130A1000227BB
:10012000861386120800AC012C08063C031C9D288F
:100130006E220130AC07031C94281F308305080091
:10014000AC012C08023C031CAA286E220130AC072B
:10015000031CA1281F308305152315236E226E2250
:1001600008006E224D233C233C233C234D236E226A
:1001700008006E228822342334233423A8226E22DE
:1001800008006E22F42297229722972297226E224D
:1001900008006E229722882297229722F4226E224C
:1001A00008006E22882234233423342334236E2221
:1001B00008006E226E229722882297226E226E22DB
:1001C00008006E225D2315239722882265236E2264
:1001D00008006E2288227423B022052388226E2212
:1001E00008006E22882215231523152315236E225D
:1001F00008006E2284233423342334238C236E227C
:1002000008006E22652365238822652365236E22FC
:1002100008006E22242305231523052324236E22A0
:1002200008006E22E4225D2315235D23E4226E2262
:1002300008006E22242315235D23152324236E2218
:1002400008006E2288223C233C233C23CA226E22D3
:1002500008006E2288223C239423342384236E22B8
:1002600008006E228822B022A822972297226E22AE
:1002700008006E229722A822B022A82297226E227E
:1002800008006E2297229C233423A42397226E22F7
:1002900008006E22F4229C233423A423F4226E222D
:1002A00008006E226E229722882215236E226E226B
:1002B00008006E22AC2334233423342384236E229B
:1002C00008006E229722342334233423A8226E227E
:1002D00008006E225D23A8228C23882205236E222B
:1002E00008006E22B42334233423342305236E22E2
:1002F00008006E22F4223423342334238C236E220C
:1003000008006E2265239C233C233C23E4226E22BA
:1003100008006E220523B4233423B42305236E2260
:1003200008006E22E42234233423342324236E2253
:1003300008006E2215230523B022742365236E2244
:1003400008006E226E226E2208007B226E227B2223
:100350006E226E226E2208007B227B227B226E227E
:100360007B227B227B226E227B226E227B226E22CC
:100370006E226E2208007B227B227B226E227B2251
:100380007B227B226E227B227B227B226E227B229F
:100390007B227B226E227B227B227B226E226E229C
:1003A0006E2208007B227B227B226E227B226E2221
:1003B0007B227B227B226E227B226E226E226E2289
:1003C00008007B226E227B227B227B226E227B22F4
:1003D0007B227B226E226E226E2208007B227B22F1
:1003E0007B226E227B226E227B226E227B227B224C
:1003F0007B226E227B226E226E226E2208007B22DE
:100400007B227B226E227B226E227B226E227B222B
:100410006E226E226E2208007B226E227B226E22CA
:100420007B226E227B227B227B226E226E226E2218
:1004300008007B226E227B227B227B226E227B2283
:100440006E227B226E226E226E2208007B226E229A
:100450007B226E227B227B227B226E226E226E22E8
:1004600008007B227B227B226E227B227B227B2246
:100470006E227B227B227B226E227B227B227B22AE
:100480006E227B226E226E226E2208006E227B225A
:100490007B227B226E227B226E227B226E226E22A8
:1004A0006E2208007B226E227B227B227B226E2220
:1004B0007B227B227B226E227B226E226E226E2288
:1004C00008007B227B227B226E227B226E227B22F3
:1004D0007B227B226E226E226E220800AE012E0845
:1004E000063C031C782ABC230130AE07031C6F2A8C
:1004F0001F3083050800AE012E08063C031C852A28
:10050000C2230130AE07031C7C2A1F30830508007C
:10051000BC23AE012E08043C031C932AC2230130E5
:10052000AE07031C8A2A1F308305BC230800BC23A6
:10053000C223AE012E08023C031CA32ABC230130B7
:10054000AE07031C9A2A1F308305C223BC23080070
:10055000BC23BC23C223BC23C223BC23BC2308006E
:10056000AE012E08023C031CBA2ABC230130AE07A0
:10057000031CB12A1F308305C223AE012E08023CA2
:10058000031CC72ABC230130AE07031CBE2A1F3040
:1005900083050800AE012E08023C031CD42ABC23AC
:1005A0000130AE07031CCB2A1F308305AE012E0895
:1005B000023C031CE02AC2230130AE07031CD72AE9
:1005C0001F308305BC230800AE012E08033C031C2A
:1005D000EE2ABC230130AE07031CE52A1F30830539
:1005E000C223C223BC230800BC23BC23AE012E08B7
:1005F000023C031C002BC2230130AE07031CF72A68
:100600001F308305BC23BC230800BC23BC23C223AA
:10061000AE012E08033C031C122BBC230130AE0795
:10062000031C092B1F3083050800BC23C223AE0125
:100630002E08043C031C212BBC230130AE07031CF5
:10064000182B1F3083050800BC23BC23AE012E08E5
:10065000033C031C302BC2230130AE07031C272BA5
:100660001F308305BC230800BC23C223BC23C22344
:10067000BC23C223BC230800AE012E08023C031C8D
:10068000462BBC230130AE07031C3D2B1F308305D6
:10069000C223BC23C223BC230800BC23AE012E0806
:1006A000033C031C582BC2230130AE07031C4F2B05
:1006B0001F308305BC23BC230800BC23BC23C223FA
:1006C000C223BC23BC23BC230800AE012E08043C7B
:1006D000031C6F2BBC230130AE07031C662B1F309D
:1006E0008305C223BC230800AE012E08033C031C73
:1006F0007E2BBC230130AE07031C752B1F308305F6
:10070000C223BC23BC230800BC23C223BC23BC23BC
:10071000C223BC23BC230800BC23BC23C223BC23AC
:10072000BC23C223BC230800BC23BC23C223C22396
:10073000BC23C223BC230800BC23C223C223BC2386
:10074000BC23C223BC230800BC23C223BC23BC237C
:10075000C223C223BC230800BC23C223C223BC2360
:10076000C223C223BC230800BC23C223BC23C22350
:10077000C223C223BC23080086110830A000A101B7
:10078000022708008615063084001030AA00FD30CC
:10079000A0000130A1000830A2000030A3003D27D6
:1007A0000800061086178616BC30A0000230A10093
:1007B0000227A52578259C25A924AC012C08013CFD
:1007C000031CE82BB224A9240130AC07031CDE2B48
:1007D0001F308305A924AC012C08013C031C012C0B
:1007E00054254B25A52578259C25422539253925D5
:1007F000A52527259C251E25A0240130AC07031C18
:10080000EC2B1F308305A02442253925A52527255B
:100810009C258125F124F1249325A52527259C25B8
:10082000E824DF246F256F25C4244225E824812590
:10083000DF2454251E25DF248125A0241E25DF2446
:10084000BB2442250C25FA24A9246F250C2542251A
:10085000BB24F1240C258125A024D624FA24A52527
:10086000932515259C2530256F25A024A0247825C7
:1008700039258125A024A525DF249C253925BB24E5
:10088000F124F124C424A024A024BB24FA24F124BC
:10089000A0243025DF248125F12454254225BB24C2
:1008A0006F25A024A525F12427255425A9249C25BE
:1008B0005425FA24CD240C25A52542259C2539252F
:1008C00039253925A52503259C25BB2481255425BB
:1008D0004225BB24C424C4245425FA240C25A52570
:1008E00003259C255425F124A024DF240325BB24C3
:1008F00054256F25A02454254B25A52578259C2516
:10090000422539253925A52566259C25BB24A52505
:100910006F259C256F2554251E25DF2481250C2558
:10092000A52503259C255425F124A924A924F430C8
:10093000A0000130A10002278613861206140800C9
:10094000C725C725C725B725C725C725B725B72577
:100950000800C725C725C725C725B725C725B7253B
:10096000B725080081259325812593258125932589
:10097000812593250800C725B725B725C725C72595
:10098000C725B725B7250800C725B725C725B7252B
:10099000C725C725B725B7250800C725B725C7250B
:1009A000B725B725C725B725B7250800C725B7251B
:1009B000B725C725B725C725B725B7250800C725FB
:1009C000B725C725C725C725C725B725B7250800DB
:1009D000C725C725C725B725C725B725B725B725F7
:1009E0000800C725C725C725C725C725B725B725AB
:1009F000B7250800C725C725C725B725B725C725AB
:100A0000B725B7250800C725C725C725B725B725AA
:100A1000B725B725B7250800C725C725C725C7258A
:100A2000B725B725B725B7250800C725B725B725AA
:100A3000B725C725B725B725B7250800C725B7258A
:100A4000C725C725B725B725B725B7250800C7256A
:100A5000B725C725B725B725B725B725B72508007A
:100A6000C725C725B725B725B725B725B725B72586
:100A70000800C725B725B725C725C725B725B7253A
:100A8000B7250800C725C725B725B725B725C7252A
:100A9000B725B7250800C725B725C725C725C7250A
:100AA000B725B725B7250800C725C725B725B7251A
:100AB000C725C725B725B7250800C725B725C725EA
:100AC000C725B725C725B725B7250800C725B725EA
:100AD000B725B725B725C725B725B7250800C725EA
:100AE000C725B725C725C725B725B725B7250800CA
:100AF000C725C725B725B725C725B725B725B725E6
:100B00000800C725C725B725C725B725C725B72599
:100B1000B7250800C725B725B725B725C725C72599
:100B2000B725B7250800C725B725C725B725C72589
:100B3000B725B725B7250800C725B725B725B72599
:100B4000B725B725B725B7250800C725B725B72589
:100B5000C725B725B725B725B7250800C725C72559
:100B6000C725C725B725B725B725B725080086159A
:100B7000063084001030AA005730A0000130A100D8
:100B80002030A2000030A3003D2786110800861502
:100B9000063084001030AA008730A0000130A10088
:100BA0001C30A2000030A3003D278611080006106B
:100BB00086178616BC30A0000230A10002277F26CF
:100BC000B7267F26B7267F26B726AC012C08013C26
:100BD000031CFF2DC5266426B7268426B726932638
:100BE000B7264826B7268926B7268926B7268D2612
:100BF000B7264D26B7260130AC07031CE62D1F3063
:100C00008305C5265726B7265426B726A526B72618
:100C10009926B7267F26B7267126C5267626B726BB
:100C20008926B7266726C5269F26B7268926C52684
:100C30004526B7265426B7266F26C5267F26B72613
:100C40005226B7266726B7266F26B7266426B7260C
:100C50004826B7264526B7267126C5267626B72606
:100C60006B26B7265226C5266726B7267626B726D0
:100C70006726B7266F26B726F430A0000130A10002
:100C800002278613861206140800DB26EE260800CB
:100C9000EE26DB26EE26DB260800EE26DB26DB260C
:100CA000DB260800DB260800EE26DB260800DB2614
:100CB000EE26EE26EE260800EE26DB26DB260800D2
:100CC000EE26DB26EE260800DB26DB260800DB26E8
:100CD000EE26DB260800DB26DB26DB260800EE26D8
:100CE0000800DB26EE26DB26DB260800DB26EE26C8
:100CF000EE26DB260800DB26DB26EE260800DB26B8
:100D0000DB26DB26EE260800EE26EE26DB26DB269B
:100D10000800DB26EE26EE260800EE26DB26DB2684
:100D2000EE26DB260800EE26EE26EE26EE26EE2642
:100D30000800DB26EE26EE26EE26EE260800DB2651
:100D4000DB26DB26EE26EE260800EE26DB26DB265B
:100D5000DB26DB260800EE26EE26EE26EE26DB2638
:100D6000080086113C30A000A1010227080086116E
:100D70003C30A000A10102273C30A000A1010227C5
:100D80003C30A000A1010227080086113C30A000E1
:100D9000A10102273C30A000A10102273C30A000A5
:100DA000A10102273C30A000A10102273C30A00095
:100DB000A1010227080086150615063084001030B0
:100DC000AA00F330A0000130A1003C30A2000030A6
:100DD000A3003D2786110611B126080086150615C9
:100DE000063084001030AA00F330A0000130A100CA
:100DF000F030A2000030A3003D2786110611B12675
:100E00000800012FA00803190D2F1427A0030000CC
:100E10000000000000000000022FA10803190800D4
:100E20001427A103A003022F0C30A500A50B162F39
:100E3000000000001230A200A20B232F2527252737
:100E400000000000080025271C2F0D30A400A40B73
:100E5000272F000008001030A8020001031C013EEB
:100E6000A902031C0800342F0A30A8020001031C49
:100E7000013EA902031C0800342F2A088004200820
:100E8000A8002108A9002B270130A202031CA303FC
:100E90002A0980052008A8002108A9002B27A208FC
:0C0EA000031D3D2FA308031D3D2F08007B
:02400E00503F21
:00000001FF
